:100000000C949E020C94E2020C94E2020C94E20224
:100010000C94E2020C94E2020C94E2020C94E202D0
:100020000C94E2020C94E2020C94060C0C94D80C92
:100030000C944A1A0C94E2020C94E2020C94E20230
:100040000C94E2020C94E2020C94E2020C94E202A0
:100050000C94E2020C94B11A0C94E2020C94E202A9
:100060000C94E2020C94E2020C94E2020C94E20280
:100070000C94E2020C94E2020C94E2020C94E20270
:100080000C94E2020C94E2020C94E2020C94E20260
:100090000C94E2020C94E2020C94E2020C94E20250
:1000A0000C94E2020C94E2020C94E2023D0D5F0D0E
:1000B0004A0E5F0D4A0EA10DC40D4A0E190E2C0EEC
:1000C00011111111401140118011E612E612E612D1
:1000D000A211E61249124912B312BB12E612E11242
:1000E00056125612561256125612561256125612D0
:1000F00056125612561256125612561256125612C0
:10010000661276127D1284128E122BA72CA42CA3B9
:10011000290014001A000800150017001C00180020
:100120000C00120013002A00002004001600070033
:1001300009000A000B000D000E000F003300340010
:10014000E1001D001B000600190005001100100051
:100150003600370038000920E000E300E20001200B
:100160000000000000000220E60065000000E4003E
:10017000000000000000000000000000000000007F
:10018000000000000000000000000000000000006F
:10019000000000000000000000000000000000005F
:1001A000000000000000000000000000000000004F
:1001B000000000000000000000000000000000003F
:1001C000000000000000000000000000000000002F
:1001D000000000000000000000000000000000001F
:1001E000000000000000000000000000000000000F
:1001F00000000000000000000000000000000000FF
:1002000000000000000000000000000000000000EE
:1002100000000000000000000000000000000000DE
:1002200000000000000000000000000000000000CE
:1002300035001E001F0020002100220023002400A2
:100240002500260027004C000100010001000100EC
:100250000100010001002D002E002F0030003100B0
:10026000010044004500680069006A006B006C00F2
:100270006D004B006F00280001000100010001002B
:1002800000000000000001004A004E0000004D0088
:1002900035021E021F022002210222022302240232
:1002A0002502260227022A00010001000100480061
:1002B0000100010001002D022E022F023002310246
:1002C00001003A003B003C003D003E003F00400082
:1002D000410042004300280001000100010001002C
:1002E0000000000000000100AB00A8000000AE000C
:1002F00000000000000000000000000000000000FE
:1003000000000000000000000000000000000000ED
:1003100000000000000000000000000000000000DD
:1003200000000000000000000000000000000000CD
:1003300000000000000000000000000000000000BD
:1003400000000000000000000000000000000000AD
:10035000000000000000000000000000000000009D
:10036000000000000000000000000000000000008D
:10037000000000000000000000000000000000007D
:10038000000000000000000000000000000000006D
:10039000000000000000000000000000000000005D
:1003A000000000000000000000000000000000004D
:1003B0002900B200B500B100B30001000100010046
:1003C000010001004600010001008350010001000E
:1003D00000500100010001000100010001000100C6
:1003E0000100010001000100010001000100010005
:1003F000010052000100280001000100010001007D
:1004000000000000000001005000510000004F00FB
:100410000A037400760034003400000006034D0027
:10042000450000000403090409025400030100A070
:10043000FA09040000010301010009211101000172
:10044000223F000705810308000A09040100010397
:100450000000000921110100012236000705820376
:1004600008000A090402000103000000092111012B
:100470000001223900070583031000011201100159
:1004800000000008EDFE606041040102000105016A
:100490000906A101050719E029E7150025019508BE
:1004A000750181020508190129059505750191025B
:1004B000950175039101050719002977150025019C
:1004C000957875018102C005010980A10185021698
:1004D000010026B7001A01002AB7007510950181A6
:1004E00000C0050C0901A1018503160100269C022C
:1004F0001A01002A9C02751095018100C0050109AE
:1005000006A101050719E029E715002501950875E1
:1005100001810295017508810105081901290595D8
:1005200005750191029501750391010507190029CF
:10053000FF150025FF950675088100C011241FBE18
:10054000CFEFDAE0DEBFCDBF04B603FE24C080915A
:10055000D8019091D901A091DA01B091DB018730E7
:10056000904BA740B04BB9F41092D8011092D9012A
:100570001092DA011092DB0114BE84B7877F84BF2A
:1005800088E10FB6F89480936000109260000FBE6F
:10059000E0E0F8E3099511E0A0E0B1E0EAE0FDE376
:1005A00002C005900D92AE32B107D9F711E0AEE26C
:1005B000B1E001C01D92A83DB107E1F70E944E09CC
:1005C0000C94831E0C94000080912F018F5F883063
:1005D00018F480932F0102C010922F0190912F01E7
:1005E00080912E01981718F4229A2A9A0895229839
:1005F0002A98089522982A980C94AF1D80932E0172
:10060000089508950895089508950E94FA020C949B
:1006100002030E9403030C94E4020C94040381E09F
:1006200008950C940F0308950F931F93CF93DF93B6
:10063000EC0108811981C8010E947B18B8010E9451
:10064000AF038C01BE010E941103882309F47AC014
:100650008A818823C9F180913B0181111EC0043138
:1006600080E5180789F50E94130381E080933B0120
:100670000E947C1A90933A018093390110923201C2
:10068000109234011092330110923601109235010C
:10069000109238011092370155C080913901909124
:1006A0003A010E94881A883C910570F480913201C9
:1006B000E82FF0E0EE0FFF1FED5CFE4F118300838B
:1006C0008F5F809332013EC0043880E5180721F027
:1006D00005381045A1F02AC08A81882321F01092A4
:1006E000300182E012C080913001811106C086E2A3
:1006F0000E94AF0F86E20E94771082E014C08A81C8
:10070000882331F01092310180E20E94C6101AC095
:1007100080913101811106C087E20E94AF0F87E20C
:100720000E94771080E20E94CD100CC081E080937F
:10073000300180933101CE01DF91CF911F910F9154
:100740000C940D0380E0DF91CF911F910F910895DC
:100750000C9405030C94090380E090E008959CE05C
:10076000799FF001112490E3899FE00DF11D112480
:10077000E60FF11DEE0FFF1FE05FFE4F8591949194
:100780000895880F991F86579040FC018591949198
:100790000895880F991F865F9E4FFC018591949163
:1007A00008950F931F93CF93DF93EC01811521E3FD
:1007B0009207A0F5811530E3930708F0D7C0883E73
:1007C0009105D8F4803E910508F06FC0883A9105F4
:1007D00078F4853A910508F06AC08130910509F4F2
:1007E000F4C108F4EFC18430910508F05EC0EAC19D
:1007F0008B3B910508F466C0E5C1C11580E2D807BE
:1008000008F0AFC0C11591E0D90708F04EC0C03F55
:10081000D10508F4D7C18E01106518C2803820E5D3
:10082000920700F5803730E5930708F0A3C0C115A3
:1008300080E5D80709F4ACC050F4CE019054803163
:100840009F4008F0BFC18E011F70106AFFC1C13008
:1008500030E5D30709F4AAC0C43180E5D80708F40D
:10086000ABC0B0C1C33890E5D90709F48EC050F4CD
:10087000C13830E5D30709F482C008F083C000E036
:1008800011EDE4C1C03191E5D90708F49BC1C11550
:1008900027E5D20708F432C1CE0190578115904167
:1008A00008F090C18E011F708BC18E01CFC1853AB7
:1008B000910509F48DC1863A910509F48CC103E8CC
:1008C00010E4C4C1883A910509F488C1893A9105B8
:1008D00009F487C18A3A910509F486C18B3A9105DA
:1008E00009F485C18C3A910509F484C18D3A9105CA
:1008F00009F483C1803B910509F482C18E3A9105C8
:1009000009F481C18F3A910509F480C1813B9105B9
:1009100009F47FC1823B910509F47EC1833B9105B7
:1009200009F47DC1843B910509F47CC1853B9105A7
:1009300009F47BC1863B910509F47AC1873B910597
:1009400009F479C1883B910509F478C1893B910587
:1009500009F477C18A3B910509F076C10AE216E4F1
:1009600075C1CE019F700E94C90371C18C0111270E
:10097000106C6CC18C010F701127146D67C100E001
:1009800010ED64C100E012ED61C100E013ED5EC145
:100990000E9450138FEF94E32CE081509040204050
:1009A000E1F700C000000E94D61A50C18091C20138
:1009B00081608093C2014AC10E94881C811102C0DB
:1009C0000E94691C0E94A51C90E09093D70180931F
:1009D000D601C23030E5D30721F48091D601816081
:1009E00086C0C43080E5D80721F48091D6018260AA
:1009F0007EC0C63090E5D90721F48091D60184608D
:100A000076C0C83020E5D20719F48091D60127C0FE
:100A1000CA3030E5D30721F48091D601806167C0E8
:100A2000CC3080E5D80721F48091D60180625FC088
:100A3000CE3090E5D90721F48091D601806457C06B
:100A4000C03120E5D20721F48091D60180684FC0E3
:100A5000C23130E5D30729F48091D60184608860E3
:100A600046C0C33080E5D80721F48091D6018E7F3F
:100A70003EC0C53090E5D90721F48091D6018D7F25
:100A800036C0C73020E5D20721F48091D6018B7F94
:100A90002EC0C93030E5D30719F48091D60126C0A5
:100AA000CB3080E5D80721F48091D6018F7E1FC01E
:100AB000CD3090E5D90721F48091D6018F7D17C004
:100AC000CF3020E5D20721F48091D6018F7B0FC073
:100AD000C13130E5D30721F48091D6018F7707C06B
:100AE000C331D04531F48091D6018B7F877F8093CD
:100AF000D6018091D6010E94A91CA8C08D2F9927EC
:100B00008F70992781309105E9F48E0103701127C8
:100B10009C0102C0220F331F0A95E2F789011C686D
:100B2000CE01E4E0880F991FEA95E1F788279370DA
:100B3000082B192BF3E0CC0FDD1FFA95E1F7C076F7
:100B4000DD272CC08230910529F41C2F0027016F6E
:100B5000106A7CC08330910561F4CE0183709927BF
:100B600001E010E002C0000F111F8A95E2F71C6837
:100B70000EC084309105A9F4CE018370992701E05D
:100B800010E002C0000F111F8A95E2F71A6863E0B7
:100B9000CC0FDD1F6A95E1F7C07ED7700C2B1D2BA3
:100BA00055C08530910529F41C2F0027046F106A69
:100BB0004DC0069709F04AC0CF71DD271C2F0027D2
:100BC000106244C000E010E041C001E010E03EC00F
:100BD00001E810E43BC002E810E438C002EE14E47F
:100BE00035C009EE14E432C00AEE14E42FC005EB60
:100BF00014E42CC006EB14E429C007EB14E426C06F
:100C00000CEC14E423C00DEC14E420C003E815E45C
:100C10001DC00AE815E41AC002E915E417C004E98A
:100C200015E414C001E216E411C003E216E40EC09C
:100C300004E216E40BC005E216E408C006E216E47E
:100C400005C007E216E402C000E014E4C801DF9129
:100C5000CF911F910F9108959CE0799FF00111248D
:100C600090E3899FE00DF11D1124E60FF11DEE0FB9
:100C7000FF1FE05FFE4F85919491803E9105E0F467
:100C8000803C910558F58133910509F46FC048F413
:100C90008932910509F463C08A32910509F46DC067
:100CA00072C089339105E9F082389105D1F085331E
:100CB000910509F44DC067C0833E910581F138F478
:100CC000803E9105B9F0823E9105D9F05CC0863E28
:100CD000910561F1873E9105A1F155C00E94C103C4
:100CE00008952091D60120FD02C021FF4CC080EE66
:100CF00090E049C08091D60180FFF9CF89E390E070
:100D000042C08091D60182FF0EC08091D60184FF3F
:100D100003C080E090E037C083EE90E034C0809163
:100D2000D60182FFF2CF82EE90E02DC08091D601F5
:100D300083FF0BC08091D60184FDEBCF87EE90E05E
:100D400022C08091D60183FFF5CF86EE90E01BC0D4
:100D50008091D60185FF07C089E290E014C08091A0
:100D6000D60185FFF9CF85E390E00DC08091D601D3
:100D700086FF07C08AE290E006C08091D60186FF18
:100D8000F9CF81E390E00E94D103089508950C9477
:100D9000C606E82FF0E0E55EFE4F8081E82FEF7099
:100DA000F0E0282F22952F7081E090E0022E01C004
:100DB000880F0A94EAF780A308950F931F93CF93A7
:100DC000DF9385B7806885BF85B7806885BFC3E03E
:100DD000D0E001E010E0FE01E55EFE4F8081E82FEB
:100DE000EF70F0E021A182958F70A80102C0440F3E
:100DF000551F8A95E2F7242B21A38C2F0E94C90648
:100E0000219748F78BE090E041E050E0FC01E15F82
:100E1000FE4F2081E22FEF70F0E062A122952F704B
:100E2000DA0102C0AA0FBB1F2A95E2F76A2B62A360
:100E3000019760F7DF91CF911F910F910C94A80358
:100E4000EF92FF920F931F93CF93DF93C4E4D1E00F
:100E500083E0E82E01E010E095E0F92E8E2D0E944F
:100E6000C9062BE030E040E050E0F901E15FFE4FC1
:100E70008081E82FEF70F0E060A170E082958F70C4
:100E800002C0759567958A95E2F760FD09C0B801C3
:100E9000022E02C0660F771F0A94E2F7462B572BEB
:100EA0002150310910F73A912A912417350721F082
:100EB00059834883F09200018E2D0E94C906EA945E
:100EC0009FEFE912CBCF8091000187FD2CC08150AC
:100ED000809300018F3F09F5809142019091430179
:100EE00090934B0180934A01809140019091410180
:100EF000909349018093480180913E0190913F0178
:100F0000909347018093460180913C0190913D016F
:100F1000909345018093440106C08FE99FE00197BB
:100F2000F1F700C000000E94AA0381E0DF91CF9199
:100F30001F910F91FF90EF900895E82FF0E0EE0FD2
:100F4000FF1FEC5BFE4F80819181089508951F93F0
:100F5000CF93DF93CCE4D1E010E09A918A910E9484
:100F6000F419180F81E0C434D807B9F7812FDF9145
:100F7000CF911F91089580915C0108950895CF93BA
:100F8000DF9300D01F92CDB7DEB72091CD01243082
:100F900021F523E029839B838A8382E08093E90003
:100FA0008FEF9091E800815095FD06C095ED9A95E0
:100FB000F1F700008111F5CF8091E80085FF0DC0A9
:100FC00040E050E063E070E0CE0101960E94F90934
:100FD0008091E8008E778093E8000F900F900F903B
:100FE000DF91CF910895CF93DF9300D01F92CDB7BB
:100FF000DEB72091CD01243019F522E029839B83AF
:101000008A832093E9008FEF9091E800815095FD4D
:1010100006C095ED9A95F1F700008111F5CF80910A
:10102000E80085FF0DC040E050E063E070E0CE01D5
:1010300001960E94F9098091E8008E778093E8007C
:101040000F900F900F90DF91CF910895CF93DF9382
:10105000EC018091CD01843009F047C080910B01F3
:101060008823E1F080910C018823C1F083E0809314
:10107000E9008FEF9091E800815095FD06C095E161
:101080009A95F1F700008111F5CF8091E80085FF76
:101090002CC040E050E060E170E017C081E0809338
:1010A000E9008FEF9091E800815095FD06C095ED25
:1010B0009A95F1F700008111F5CF8091E80085FF46
:1010C00014C040E050E068E070E0CE010E94F909F1
:1010D0008091E8008E778093E80080E1FE01ACE427
:1010E000B1E001900D928A95E1F7DF91CF910895DB
:1010F0008091CC01811109C00E948B0B0E94E80BEA
:101100008091E20084608093E20008951092CC0107
:101110000895089508950C943F1A42E061EC81E02F
:101120000E94050B42E061EC82E00E94050B42E167
:1011300061EC83E00C94050B8091CF01833009F4BE
:1011400055C030F4813071F0823009F48EC00895BA
:101150008A3009F47AC08B3009F460C0893009F014
:101160009CC020C08091CE01813A09F096C0809148
:10117000E800877F8093E8008091D2019091D301AD
:10118000892B21F060E080E090E003C060E18CE416
:1011900091E070E00E94420A8091E8008B77809392
:1011A000E80008958091CE01813209F076C08091E7
:1011B000D2019091D301009719F0029709F06DC008
:1011C0008091E800877F8093E8008091E80082FDAD
:1011D00005C08091CD018111F8CF5FC08091F100F1
:1011E00080935C018091E8008B7753C08091CE01A1
:1011F000813A09F052C08091D2019091D301892B9C
:1012000009F04BC08091E800877F8093E8008091CF
:10121000E80080FFFCCF80910B0136C08091CE01A9
:101220008132D9F58091D2019091D301892BA9F512
:101230008091E800877F8093E8000E943A0B8091BC
:10124000D00180930B010C9450138091CE01813218
:1012500021F58091E800877F8093E8000E943A0B97
:101260008091D10180935D0108958091CE01813AF2
:10127000A1F48091E800877F8093E8008091E800E6
:1012800080FFFCCF80915D018093F1008091E800A8
:101290008E778093E8000C943A0B089584B7877F8B
:1012A00084BF88E10FB6F8948093600010926000CC
:1012B0000FBE90E080E80FB6F894809361009093A1
:1012C00061000FBE0E94C90E0E948B0B0E94E80BAA
:1012D0008091E20084608093E20078940E94630E23
:1012E0000E94CB0E81E091E00E94800E8091CD01A2
:1012F000853069F40E94001A8091CB018823B1F3F4
:101300000E942E1A882391F30E94E309EFCF0E94D6
:10131000D30EECCF292F332723303105A9F06CF4FD
:101320002130310509F442C02230310509F043C0B3
:1013300084E590E028E234E042C021323105C9F072
:101340002232310519F137C099278130910541F0DA
:101350008230910541F0892B71F5E4E2F4E005C09B
:10136000ECE1F4E002C0E0E1F4E0849190E09F0160
:1013700026C0633000F5E62FF0E0EE0FFF1FE85DBA
:10138000FE4F2081318189E090E019C0633098F4EC
:10139000E62FF0E0DF01AA0FBB1FAE5DBE4F2D911F
:1013A0003C91E15EFE4F808190E009C082E190E0D7
:1013B0002CE734E004C080E090E020E030E0FA0167
:1013C00031832083089580E189BD82E189BD09B41C
:1013D00000FEFDCF8091D8008F7D8093D800809152
:1013E000E00082608093E0008091E00081FDFCCF0E
:1013F0000895CF92DF92EF92FF920F931F93CF93B6
:10140000DF937C018B01EA010E945B0B811131C0EB
:10141000209731F088819981081B190BE80EF91E7D
:10142000C12CD12C0115110519F18091E80085FD21
:1014300014C08091E8008E778093E800209741F0F7
:10144000888199818C0D9D1D9983888385E011C0C9
:101450000E945B0B882331F30CC0F70181917F015F
:101460008093F10001501109FFEFCF1ADF0ADACFA4
:1014700080E0DF91CF911F910F91FF90EF90DF906F
:10148000CF9008952091D4013091D50126173707C8
:1014900048F06115710539F42091E8002E7720930A
:1014A000E80001C0B901FC0120E061157105B9F146
:1014B0008091CD01882309F440C0853009F43FC0F4
:1014C0008091E80083FD3DC08091E80082FF06C066
:1014D0008091E80082FF26C080E008958091E800B6
:1014E00080FFE3CF2091F3008091F20090E0922BF7
:1014F0006115710551F08830910538F421912093E0
:10150000F100615071090196F3CF21E0089709F0CD
:1015100020E08091E8008E778093E800C6CF21110B
:10152000C7CFD6CF8091CD01882339F0853039F0EF
:101530008091E80083FFCCCF04C082E0089583E06F
:10154000089581E008952091D4013091D5012617A6
:10155000370748F06115710539F42091E8002E77BE
:101560002093E80001C0B901FC0120E0611571057C
:10157000C1F18091CD01882309F441C0853009F47F
:1015800040C08091E80083FD3EC08091E80082FF6A
:1015900006C08091E80082FF27C080E00895809116
:1015A000E80080FFE3CF2091F3008091F20090E00B
:1015B000922B6115710559F08830910540F4249102
:1015C0002093F1003196615071090196F2CF21E02C
:1015D000089709F020E08091E8008E778093E8007A
:1015E000C5CF2111C6CFD5CF8091CD01882339F049
:1015F000853039F08091E80083FFCBCF04C082E0D2
:10160000089583E0089581E00895982F973058F564
:101610009093E900981739F07091EC002091ED005B
:101620005091F00003C0242F762F50E021FF19C005
:101630003091EB003E7F3093EB003091ED003D7F29
:101640003093ED003091EB0031603093EB007093FC
:10165000EC002093ED005093F0002091EE0027FF66
:1016600007C09F5FD3CF8F708093E90081E008951A
:1016700080E008958091CE0187FD05C08091E8004B
:1016800080FF0EC012C08091E80082FD05C08091ED
:10169000CD018111F8CF08958091E8008B7708C0C3
:1016A0008091CD018111EACF08958091E8008E7775
:1016B0008093E80008958091E4009091E50045E66C
:1016C0002091EC0020FF21C02091E80020FD21C0E6
:1016D0002091CD01222389F0253089F02091EB0063
:1016E00025FD0FC02091E4003091E500281739074F
:1016F00039F3415041F0C901E3CF82E0089583E01E
:10170000089581E0089584E008952091E80022FF83
:10171000DFCF80E008950E94F90B0E94010CE0EEFB
:10172000F0E0808181608083E8EDF0E080818F7758
:10173000808319BCA7EDB0E08C918E7F8C93808163
:101740008F7E80831092CC0108950F931F93CF93C7
:10175000DF930E94F90B0E94010CC8EDD0E0888154
:101760008F77888388818068888388818F7D88834C
:1017700019BC1092CD011092C9011092CB011092A8
:10178000CA0100EE10E0F80180818B7F80838881A0
:101790008160888342E060E080E00E94050BE1EE1A
:1017A000F0E080818E7F8083E2EEF0E080818160D6
:1017B0008083808188608083F80180818E7F808330
:1017C000888180618883DF91CF911F910F91089567
:1017D000E8EDF0E080818F7E8083E7EDF0E08081AE
:1017E0008160808384E082BF81E08093CC010C948F
:1017F000A50BE8EDF0E080818E7F80831092E200FF
:1018000008951092DA001092E10008951F920F924D
:101810000FB60F9211242F933F934F935F936F93C3
:101820007F938F939F93AF93BF93EF93FF93809199
:10183000E10082FF0BC08091E20082FF07C080912F
:10184000E1008B7F8093E1000E94620E8091DA00BC
:1018500080FF1FC08091D80080FF1BC08091DA00FC
:101860008E7F8093DA008091D90080FF0DC080E1E7
:1018700089BD82E189BD09B400FEFDCF81E080937E
:10188000CD010E94780805C019BC1092CD010E94BC
:1018900086088091E10080FF19C08091E20080FFFE
:1018A00015C08091E2008E7F8093E2008091E2007B
:1018B00080618093E2008091D80080628093D8009C
:1018C00019BC85E08093CD010E948A088091E100D7
:1018D00084FF30C08091E20084FF2CC080E189BD8C
:1018E00082E189BD09B400FEFDCF8091D8008F7DD3
:1018F0008093D8008091E1008F7E8093E1008091F9
:10190000E2008F7E8093E2008091E200816080930C
:10191000E2008091C901882311F084E007C0809122
:10192000E30087FF02C083E001C081E08093CD0126
:101930000E948B088091E10083FF29C08091E20022
:1019400083FF25C08091E100877F8093E10082E0E2
:101950008093CD011092C9018091E1008E7F809328
:10196000E1008091E2008E7F8093E2008091E200AE
:1019700080618093E20042E060E080E00E94050B1D
:101980008091F00088608093F0000E948908FF91A8
:10199000EF91BF91AF919F918F917F916F915F91E7
:1019A0004F913F912F910F900FBE0F901F90189560
:1019B0001F920F920FB60F9211242F933F934F93C4
:1019C0005F936F937F938F939F93AF93BF93CF93C7
:1019D000EF93FF93C091E900CF708091EC001092DB
:1019E000E9008091F000877F8093F00078940E9456
:1019F000140D1092E9008091F00088608093F0004F
:101A0000C093E900FF91EF91CF91BF91AF919F916A
:101A10008F917F916F915F914F913F912F910F9097
:101A20000FBE0F901F9018951F93CF93DF93CDB7E4
:101A3000DEB7AA970FB6F894DEBF0FBECDBFEEECAF
:101A4000F1E08091F100819321E0E63DF207C9F7D2
:101A50000E949C088091E80083FF1CC12091CE0168
:101A60003091CF01832F90E08A30910508F012C1A8
:101A7000FC01EA5AFF4F0C94471E203881F02238AF
:101A800009F008C18091D2018F708093E9008091A4
:101A9000EB0085FB882780F91092E90006C0809151
:101AA000CA019091CB01911182609091E800977FDB
:101AB0009093E8008093F1001092F100C5C0822F4E
:101AC0008D7F09F0E7C0222319F0223061F0E2C0D7
:101AD0008091D001813009F0DDC0333009F080E021
:101AE0008093CB0128C08091D001811124C0209126
:101AF000D2012F7009F4CEC02093E9008091EB0051
:101B000080FF19C08091EB00333011F4806211C066
:101B100080618093EB0081E090E0022E01C0880F8D
:101B20000A94EAF78093EA001092EA008091EB00B1
:101B300088608093EB001092E9008091E800877F35
:101B400086C02111A7C01091D0011F778091E300BA
:101B50008078812B8093E3008091E800877F8093D9
:101B6000E8000E943A0B8091E80080FFFCCF809152
:101B7000E30080688093E300112311F083E001C04B
:101B800082E08093CD0186C02058223008F082C0C8
:101B90008091D0019091D1018C3D23E0920779F59D
:101BA00083E08A838AE289834FB7F894DE01139633
:101BB00020E03EE051E2E32FF0E050935700E49143
:101BC00020FF03C0E295EF703F5FEF708E2F90E033
:101BD000EA3010F0C79601C0C0968D939D932F5F99
:101BE000243149F74FBF8091E800877F8093E80058
:101BF0006AE270E0CE0101960E94420A14C0AE0172
:101C00004F5F5F4F6091D2010E948A09009709F4EB
:101C100041C02091E800277F2093E800BC01898122
:101C20009A810E94A30A8091E8008B778093E80054
:101C300031C0203879F58091E800877F8093E800F3
:101C40008091C9018093F1008091E8008E778093A4
:101C5000E8000E943A0B1EC021111CC09091D001D7
:101C60009230C0F48091E800877F8093E8009093E1
:101C7000C9010E943A0B8091C901811104C0809171
:101C8000E30087FF02C084E001C081E08093CD01C2
:101C90000E948D088091E80083FF0AC08091E800CF
:101CA000877F8093E8008091EB0080628093EB0057
:101CB000AA960FB6F894DEBF0FBECDBFDF91CF91CD
:101CC0001F9108950895CF938091CD018823B1F09D
:101CD0008091E9008F709091EC0090FF02C090E835
:101CE00001C090E0C92FC82B1092E9008091E80054
:101CF00083FD0E94140DCF70C093E900CF91089529
:101D000090936301809362010895E0916201F091E4
:101D10006301309721F00190F081E02D099480E07B
:101D20000895E0916201F0916301309721F0028003
:101D3000F381E02D099408952091600130916101B3
:101D40008217930771F09093610180936001E09195
:101D50006201F0916301309721F00680F781E02D58
:101D60000994089520915E0130915F0182179307D5
:101D700071F090935F0180935E01E0916201F091B8
:101D80006301309721F00084F185E02D09940895D6
:101D900008950C94C80E0E94731A0E94DD060E94DA
:101DA0003E1B0C94AF1D5F926F927F928F929F9219
:101DB000AF92BF92CF92DF92EF92FF920F931F9359
:101DC000CF93DF9300D000D01F92CDB7DEB70E9433
:101DD00020079DE6C92E91E0D92E03E010E0AA2449
:101DE000A394B12C502E802F0E949D073C01F60138
:101DF000F290E2906F01E826F926E114F104A1F4D3
:101E00000150110978F78FEF89838A831B820E9422
:101E10007C1A8160782F9D838C8349815A816B81E4
:101E20008D810E94810F38C08091C20181FD0E9486
:101E3000A6072BE030E04501022E02C0880C991C59
:101E40000A94E2F7C4018E219F21892B09F129838D
:101E50005A826820792081E0672809F480E08B832A
:101E60000E947C1A8160782F9D838C8349815A81DE
:101E70006B818D810E94810FF801EE0FFF1FEB59DE
:101E8000FE4F80819181882599259183808304C0AC
:101E90002150310980F6B4CF109164010E94850E63
:101EA0001817D1F00E94850E809364010F900F9057
:101EB0000F900F900F90DF91CF911F910F91FF9096
:101EC000EF90DF90CF90BF90AF909F908F907F90DA
:101ED0006F905F900C94C7060F900F900F900F902B
:101EE0000F90DF91CF911F910F91FF90EF90DF90B6
:101EF000CF90BF90AF909F908F907F906F905F90AA
:101F00000895CF93DF93CDB7DEB72B970FB6F89434
:101F1000DEBF0FBECDBF4F83588769877A878B8717
:101F2000DE01119686E0FD0111928A95E9F785E0C0
:101F3000FE01379601900D928A95E1F749815A8109
:101F40006B817C818D819E810E9420162B960FB61D
:101F5000F894DEBF0FBECDBFDF91CF910895CF9330
:101F6000C82F882309F4C1C0823859F40E94850E15
:101F700081FDBBC089E30E94FB180E94C51989E35B
:101F80000CC0833879F40E94850E80FDAEC083E5D5
:101F90000E94FB180E94C51983E50E943B19CF914E
:101FA0000C94C519843859F40E94850E82FD9DC099
:101FB00087E40E94FB180E94C51987E4EECF8CEFDE
:101FC0008C0F813A48F48C2F0E94701D81118DC0B6
:101FD0008C2F0E94FB18E3CF80E28C0F883048F4EE
:101FE000C77081E001C0880FCA95EAF70E947C198A
:101FF000D6CF8BE58C0F833078F4C53A29F0C63AFA
:1020000031F482E890E005C081E890E002C083E806
:1020100090E0CF910C949C0E88E58C0F833108F0F2
:1020200064C0C83A39F1C93A41F1CA3A49F1CB3AE8
:1020300051F1CC3A59F1CD3A61F1C03B69F1CE3A58
:1020400071F1CF3A79F1C13B81F1C23B89F1C33BD8
:1020500091F1C43B99F1C53BA1F1C63BA9F1C73B46
:10206000B1F1C83BB9F1C93BC1F1CA3BC9F58AE23C
:1020700092E038C082EE90E035C089EE90E032C048
:102080008AEE90E02FC085EB90E02CC086EB90E0CC
:1020900029C087EB90E026C08CEC90E023C08DEC4B
:1020A00090E020C083E891E01DC08AE891E01AC06A
:1020B00082E991E017C084E991E014C081E292E0E6
:1020C00011C083E292E00EC084E292E00BC085E290
:1020D00092E008C086E292E005C087E292E002C08A
:1020E00080E090E0CF910C94B20ECF9108958823B8
:1020F00009F44BC0823859F40E94850E81FF45C017
:1021000089E30E94FB180E94C51989E30CC083383B
:1021100071F40E94850E80FF38C083E50E94FB1891
:102120000E94C51983E50E943B190C94C519843897
:1021300059F40E94850E82FF28C087E40E94FB1894
:102140000E94C51987E4EFCF9CEF980F913A58F39E
:1021500090E2980F983050F4877091E001C0990F89
:102160008A95EAF7892F0E948219DFCF9BE5980FA5
:10217000933020F480E090E00C949C0E885A8331D8
:1021800020F480E090E00C94B20E0895882321F0B2
:102190000E947C190C94C5190895882321F00E948F
:1021A00082190C94C51908958F929F92AF92BF9295
:1021B000CF92DF92EF92FF920F931F93CF93DF9313
:1021C0001F92CDB7DEB74C01A62E472FFC01E5804C
:1021D000E2948FE0E822F280FF2021F079830E94D0
:1021E0009919498149830E94F4184981882381F013
:1021F000FF2071F080E28A0D883050F082E00E946A
:10220000DD180E94F418BB24B394B826498101C09C
:10221000B12CE42FE295EF70F0E0E05AFF4F0C9400
:10222000471E842F807F142F1F70882311F0129572
:10223000107FFF2089F0112309F48BC180E28A0D01
:10224000883020F4812F0E947C1903C0812F0E94C6
:102250008C190E94C5197DC18A2D0E947710112307
:1022600009F4B4C180E28A0D883020F4812F0E94E5
:10227000821903C0812F0E9492190E94C519A6C11C
:10228000242F207F842F8F70203211F08295807F41
:10229000AA2021F0F1E0AF16B1F021C0FF2041F0FB
:1022A000EE2039F191E0E91224C00E94AC198EC1F0
:1022B000EE2021F0E1E0EE1609F488C189830E9446
:1022C000AF19898100C1FF2029F0F5E0FE1508F45F
:1022D0007DC10FC094E09E1508F478C1F4C0FF20C2
:1022E00059F0EE2031F0F401958190FF32C19F70DA
:1022F00095830E94C6106AC1EE2009F4E4C02FC184
:10230000242F26952695237030E02115310521F0E4
:102310002130310561F05AC1FF2021F08A2D942F20
:10232000937002C080E090E00E949C0E4FC1FF209D
:1023300021F08A2D942F937002C080E090E00E94DB
:10234000B20E44C1842F837009F04EC0F1103EC11B
:102350002A2D229526952770220F220F8A2D8F7005
:10236000C82ED12CE12CF12C022E04C0CC0CDD1C8B
:10237000EE1CFF1C0A94D2F7A4FE10C06FE070E0C0
:1023800080E090E004C0660F771F881F991F2A9590
:10239000D2F7609570958095909503C060E070E0ED
:1023A000CB01242F26952695237030E0223031056D
:1023B00069F02330310589F06C297D298E299F2908
:1023C0002130310571F00E94721700C16C297D29FE
:1023D0008E299F290E948C17F9C00E947217C7018D
:1023E000B6010E945817F2C0FF2019F0842F8170A7
:1023F00001C08695882309F4E9C02A2D22952695E7
:102400002770220F220F8A2D8F70C82ED12CE12C1D
:10241000F12C022E04C0CC0CDD1CEE1CFF1C0A9417
:10242000D2F7A4FE10C06FE070E080E090E004C03E
:10243000660F771F881F991F2A95D2F760957095B0
:102440008095909503C060E070E0CB01242F269525
:102450002695237030E02230310569F023303105B4
:1024600089F06C297D298E299F292130310571F051
:102470000E944618ABC06C297D298E299F290E9495
:102480006018A4C00E944618C701B6010E942C180B
:102490009DC00A2D10E0F801E05EF109E531F1057B
:1024A00008F053C0E059FF4F0C94471E1A2D1F70BF
:1024B000842F8F71FF2021F00E94C517812F19CF23
:1024C0000E94E617812F0E94CD1080C0FF2049F0A6
:1024D000F4E0FE1508F47AC0842F8F710E940B1867
:1024E00075C085E08E1508F471C0F6CFFF2039F075
:1024F000842F8F710E94C51769C0FF20C9F3842FF4
:102500008F710E94E61762C0FF2029F0842F8F711F
:102510000E94B0175BC00E94A61758C0FF2051F060
:10252000142F1F71812F0E94C51763E0812F0E9415
:10253000D4184CC081E00E94DD1891E09E1508F08F
:1025400045C082E00E94DD1841C0FF2031F0EE203E
:1025500079F28A2D0E94AF0F39C0EE2081F28A2DC8
:102560000E94771033C04F706A2DC4010E94AC03E3
:102570000E94CD162BC0F11029C0942F9F70492FB7
:1025800050E042305105B9F04CF44115510581F04D
:1025900041305105D9F40E94D71D18C04330510570
:1025A00069F04430510591F48A2D0E942B1E0EC013
:1025B0000E94C01D0BC00E94F31D08C00E94061E91
:1025C00005C04F706A2DC4010E940103BB20F1F0C9
:1025D0000E94D01880FD1AC0F40112820E94CA180D
:1025E0000E94C517C4010E9414130E94CA180F90BC
:1025F000DF91CF911F910F91FF90EF90DF90CF90DF
:10260000BF90AF909F908F900C94E6170F90DF9142
:10261000CF911F910F91FF90EF90DF90CF90BF90DF
:10262000AF909F908F9008950F931F93CF93DF9358
:10263000EC01288139818B819C81892B31F03F3FCE
:1026400011F080E003C02F3FE1F781E0811113C05A
:10265000CE010E941403882371F0688179818A81F8
:102660000E94C6188C010E947A180E944D17B8016A
:10267000CE010E94D410DF91CF911F910F91089548
:102680000E9499190E94A9190E946E190E94C519E9
:1026900080E090E00E949C0E80E090E00C94B20EEE
:1026A0000E9489190C9440130E94BB18292F22956F
:1026B0002F7030E02C3031054CF42A3031056CF4A9
:1026C0002250310922303105B0F407C02C303105D9
:1026D00071F02F30310559F00EC0803F31F018F401
:1026E000803E48F402C0843F31F481E0089593FBBA
:1026F000882780F9089580E00895CF93DF9300D074
:1027000000D01F92CDB7DEB70F900F900F900F90B3
:102710000F90DF91CF910895CF93DF9300D000D039
:1027200000D0CDB7DEB726960FB6F894DEBF0FBE49
:10273000CDBFDF91CF9108951F93CF93DF93C091C9
:102740006D0116E080916E01C81799F0D0E01C9FD2
:10275000F0011D9FF00D1124E159FE4F4081518180
:1027600062817381848195810E948C132196C77048
:10277000E9CFDF91CF911F91089540919F01509132
:10278000A0016091A1017091A2018091A30190919B
:10279000A4010C948C13CF938091A40182958F7027
:1027A00009F05FC08091A101882309F45AC02091EB
:1027B0006D01A0916E0160919F017091A0018091C7
:1027C000A2019091A30131E06F3F09F030E0B32FF7
:1027D000C6E02A1709F445C0009721F07F3F21F495
:1027E0004B2F03C041E001C040E030E040FD35C068
:1027F000C29FF001C39FF00D1124E159FE4F4181AA
:1028000074132BC04081641328C04281411125C03C
:10281000438154814817590710F441505109481B0E
:10282000590B483C5105C8F48091A4018F70806118
:102830008093A40186E0829FF001839FF00D112414
:10284000EC58FE4F80818F70806180838FE991E02A
:102850000E941413CF910C949C132F5F3F4F27704D
:10286000B8CFCF910895CF92DF92EF92FF920F935E
:102870001F93CF93DF93CDB7DEB762970FB6F8946F
:10288000DEBF0FBECDBF8C0185E0F801DE011D96D5
:1028900001900D928A95E1F7D8014C9111965C91C7
:1028A000119712966C9112971396ED90FC901497D5
:1028B00070919F01E091A0012091A2013091A301AC
:1028C0002115310531F0EF3F31F481E07F3F19F4FC
:1028D00003C081E001C080E0B82FB170CB2E80FD35
:1028E0006CC1D090A101DD2009F4F5C0F091A401E4
:1028F000E216F30638F0C701821B930B883C910562
:1029000048F09BC0209530952E0D3F1D283C310589
:1029100008F093C08F2F807F09F052C0E51314C0D8
:10292000741312C0D62E61110FC0FF70F061F093C6
:10293000A4010E94BD138FE991E00E9414138091BD
:10294000A401F80185836CC1EF2831F05F3F31F4B9
:1029500081E04F3F19F403C081E001C080E080FDB9
:1029600003C081E0862701C080E0F82FF170FF2EC0
:1029700080FF1CC080916D0120916E0136E08217AE
:1029800009F428C190E0389FF001399FF00D11241F
:10299000E159FE4F7181571306C07081471303C080
:1029A0007281671303C001968770E9CFD62E662324
:1029B00009F436C18091A40181608093A40153C0C1
:1029C000E51308C0741306C0611104C0D801159640
:1029D000FC93AEC04D875E878D859E856A8B0E9475
:1029E00054136A89882329F1D62E662311F1209188
:1029F000A401822F82958F7090E002970CF460C042
:102A000080919F019091A00198878F831986FB8602
:102A1000EA862C87CE01079651C0E51731F14D8724
:102A20005E878D859E856A8B0E9454136A89811109
:102A30002EC0C8010E941413A4C08F2F807F69F795
:102A40007E2DF98AE88A89890E947D138FE991E0B9
:102A50000E941413EFE9F1E086E0DF011D928A95F0
:102A6000E9F70E94BD13D12CDBC07413D8CF6111DC
:102A7000D6CFD8011596FC93C8010E941413EFE934
:102A8000F1E086E0DF011D928A95E9F7C9C0D62EF4
:102A9000662379F22091A401822F82958F7090E0B5
:102AA000029774F080919F019091A0019A8389838D
:102AB0001B82FD82EC822E83CE0101960E941413AC
:102AC00086E0F801AFE9B1E001900D928A95E1F757
:102AD0000E94CB136FC0E216F30628F0C701821BD9
:102AE000930B9C0104C0209530952E0D3F1D283C72
:102AF000310508F052C0D62E662309F49ACFE513AB
:102B00002CC074132AC08091A40180FD1DC0982F91
:102B100092959F70C9F0D80115968C9315979F30A8
:102B200039F09F5F9295907F8F70892B15968C93CB
:102B3000C8010E94141386E0F801AFE9B1E00190EA
:102B40000D928A95E1F736C086E0F801AFE9B1E071
:102B500001900D928A95E1F763C04D875E878D8560
:102B60009E850E945413882379F086E0F801AFE92E
:102B7000B1E001900D928A95E1F70E94CB130E947B
:102B8000BD13DD24D3944CC08091A4018160809357
:102B9000A401C8010E94141343C07E2DF98AE88A5B
:102BA00089890E947D13EFE9F1E086E0DF011D9243
:102BB0008A95E9F70E94BD1333C0662309F439CF23
:102BC0004D875E878D859E850E945413882309F466
:102BD00030CFCBCF4D875E878D859E850E94BB18F9
:102BE000292F22952F7030E0223031052CF49F7070
:102BF00041F0811106C00CC0243031052CF49F70C7
:102C000049F4805E883020F0C8010E941413CF2C54
:102C1000DC2C06C0D80115969C91907F91F7F8CFD7
:102C20008D2D62960FB6F894DEBF0FBECDBFDF913B
:102C3000CF911F910F91FF90EF90DF90CF9008956B
:102C40001F93CF93DF93CDB7DEB72C970FB6F894D1
:102C5000DEBF0FBECDBF4F83588769877A878B87CA
:102C60009C87CE0107960E9433148823C1F02F81E0
:102C700038858A859B85892B31F03F3F11F080E0B4
:102C800003C02F3FE1F781E0811147C04F81588594
:102C900069857A858B859C850E948C133EC086E071
:102CA000FE013796DE01119601900D928A95E1F7AB
:102CB000FF81E8854A855B854115510531F0EF3F7D
:102CC00031F481E0FF3F19F403C081E001C080E0EE
:102CD00080FD23C020916E0130E0C901019687700C
:102CE000992760916D0170E086179707F1F1F983DC
:102CF000EA835D834C8396E0929FD001939FB00D51
:102D00001124A159BE4FFE01319601900D929A9562
:102D1000E1F780936E010E949C1316E080916D0193
:102D200090916E01891779F1189FC0011124815982
:102D30009E4F0E943314882331F1E0916D011E9F54
:102D4000F0011124E159FE4F40815181628173816C
:102D5000848195810E948C1380916D0190E0019691
:102D60008770992780936D01D9CF0E9450131092DC
:102D70006E0110926D01EFE9F1E086E0DF011D9236
:102D80008A95E9F7CACF2C960FB6F894DEBF0FBE2E
:102D9000CDBFDF91CF911F910895EF92FF920F93D6
:102DA0001F93CF93DF93FC01009709F46FC0F12CC0
:102DB000EE24E394EF0121968491843740F484302B
:102DC00008F055C0813081F0823021F15FC0853735
:102DD00009F447C0C0F19CE7980F903708F056C03F
:102DE0008F770E94771045C08F010E5F1F4FFE0145
:102DF000849190E2980F983050F48770FE2D01C0B6
:102E0000FF0F8A95EAF78F2F0E949C1915C00E9428
:102E1000AF0F14C08F010E5F1F4FFE01849190E22F
:102E2000980F983068F48770FE2D01C0FF0F8A95C7
:102E3000EAF78F2F0E94A2190E94C519E80119C054
:102E40000E947710FBCFCF010296FE01C491CC23E4
:102E500061F0EFE9FFE03197F1F700C00000C150E9
:102E6000F6CFCF010296FE01F490EC0102C00E9461
:102E7000AF0F8F2D882341F0EFE9FFE03197F1F795
:102E800000C000008150F6CFFE0194CFDF91CF91BA
:102E90001F910F91FF90EF90089508956093A901FD
:102EA0007093AA018093AB019093AC010C944013F2
:102EB0000F931F930091A9011091AA012091AB01DA
:102EC0003091AC01062B172B282B392B0093A9012D
:102ED0001093AA012093AB013093AC011F910F9185
:102EE0000C9440130F931F930091A9011091AA0114
:102EF0002091AB013091AC010623172328233923FD
:102F00000093A9011093AA012093AB013093AC0167
:102F10001F910F910C9440130F931F930091A901DF
:102F20001091AA012091AB013091AC01062717271F
:102F3000282739270093A9011093AA012093AB01F8
:102F40003093AC011F910F910C9440131092A50186
:102F50001092A6011092A7011092A8010C944013A0
:102F600041E050E060E070E004C0440F551F661F70
:102F7000771F8A95D2F74093A5015093A6016093DD
:102F8000A7017093A8010C94401341E050E060E069
:102F900070E004C0440F551F661F771F8A95D2F753
:102FA0008091A5019091A601A091A701B091A801DF
:102FB000842B952BA62BB72B8093A5019093A6016C
:102FC000A093A701B093A8010C94401341E050E0F6
:102FD00060E070E004C0440F551F661F771F8A959C
:102FE000D2F740955095609570958091A50190918C
:102FF000A601A091A701B091A80184239523A6233F
:10300000B7238093A5019093A601A093A701B09345
:10301000A8010C94401341E050E060E070E004C06F
:10302000440F551F661F771F8A95D2F78091A5011F
:103030009091A601A091A701B091A801842795279E
:10304000A627B7278093A5019093A601A093A70177
:10305000B093A8010C9440130F931F930091A50106
:103060001091A6012091A7013091A801062B172BE2
:10307000282B392B0093A5011093A6012093A701BB
:103080003093A8011F910F910C9440130F931F933D
:103090000091A5011091A6012091A7013091A801EE
:1030A00006231723282339230093A5011093A60193
:1030B0002093A7013093A8011F910F910C94401306
:1030C0000F931F930091A5011091A6012091A701D4
:1030D0003091A80106271727282739270093A50133
:1030E0001093A6012093A7013093A8011F910F917F
:1030F0000C9440130895CF92DF92EF92FF920F93BA
:103100001F93CF93DF93EC01C090A901D090AA0147
:10311000E090AB01F090AC018091A5019091A601E7
:10312000A091A701B091A801C82AD92AEA2AFB2AAE
:103130000FE110E0B701A601002E04C07695679557
:10314000579547950A94D2F740FD05C001501109E3
:1031500088F780E007C0BE01802F0E942C060197EF
:10316000A9F3802FDF91CF911F910F91FF90EF90E6
:10317000DF90CF900895CF93DF93EC010E947B18EE
:10318000BE010E942C06DF91CF910895CB010E94D1
:10319000BB1808958091AD01859585958595089515
:1031A0008091AD018770089598E0899F9001112466
:1031B000622B6093AD010C94C5174091AD018095D1
:1031C00084238093AD01982F977069F450E0282FE5
:1031D000332727FD30954217530729F085958595AC
:1031E00085950C94E61708959091AD01977081E054
:1031F00009F480E0089590910B019923D9F0909102
:103200000C019923B9F0982F9695969596959F3035
:1032100088F5E0910D01F0910E01E90FF11D877025
:1032200021E030E001C0220F8A95EAF78181822BEC
:103230008183089540910D0150910E0120E030E00E
:103240009FEFFA01E20FF31F6281681799F09F3F29
:1032500019F4611101C0922F2F5F3F4F2E303105BD
:1032600081F79F3F39F0FA01E90FF11D97FDFA95BB
:1032700082830895089590910B019923E1F0909134
:103280000C019923C1F0982F9695969596959F30AD
:1032900020F5E0910D01F0910E01E90FF11D87700D
:1032A00021E030E001C0220F8A95EAF72095818164
:1032B00028232183089540910D0150910E0120E0B3
:1032C00030E0FA01E20FF31F9281981301C01282DD
:1032D0002F5F3F4F2E303105A1F7089581E090E038
:1032E000E0910D01F0910E01E80FF91F1082019697
:1032F00080319105A9F708959091C101982B909381
:10330000C101089580959091C10198239093C101C6
:1033100008951092C10108959091C001982B909347
:10332000C001089580959091C00198239093C001A9
:1033300008951092C00108959091BF01982B909329
:10334000BF01089580959091BF0198239093BF018C
:1033500008951092BF0108958093AE0108951092D0
:10336000AE01089540910D0150910E0120E030E032
:1033700080E0FA01E20FF31F918191118F5F2F5FBF
:103380003F4F2F303105A9F70895E0910D01F091DD
:103390000E018091C1018083E0910D01F0910E0139
:1033A00080819091C001892B8083E0910D01F09183
:1033B0000E0180819091BF01892B80839091AE0195
:1033C000992361F0E0910D01F0910E018081892B2C
:1033D00080830E94B21981111092AE0180910D017B
:1033E00090910E010C94910E40E0009739F09C01F1
:1033F00021503109822393234F5FF7CF842F089503
:103400008091CD01843039F11092C30120E488E12C
:1034100090E00FB6F894A895809360000FBE2093BB
:10342000600080E00E94FE0280E00E94C70683B731
:10343000817F846083BF83B7816083BF78948895E0
:1034400083B78E7F83BF88E10FB6F89480936000C6
:10345000109260000FBE08950895089580E00E94C4
:10346000FE020E942C1A0E9420070E942D1A0E9420
:10347000A70791E0811101C090E0892F08950E9473
:10348000501380E00E94FE020E94AF1D0E94850E34
:103490000C94C7061F920F920FB60F9211248F93B0
:1034A0009F93AF93BF938091C301811113C080910B
:1034B000C4019091C501A091C601B091C701419688
:1034C000A11DB11D8093C4019093C501A093C601B5
:1034D000B093C701BF91AF919F918F910F900FBE95
:1034E0000F901F90189582E084BD93E095BD9AEFF0
:1034F00097BD80936E0008952FB7F8948091C40112
:103500009091C501A091C601B091C7012FBF089548
:10351000CF92DF92EF92FF920F931F932FB7F89401
:103520004091C4015091C5016091C6017091C701DD
:103530002FBF6A017B01EE24FF248C0120E030E0E4
:10354000C016D106E206F30610F441505109481B9B
:10355000590BCA011F910F91FF90EF90DF90CF9010
:1035600008951F920F920FB60F9211248F939F937D
:10357000AF93BF938091C4019091C501A091C60102
:10358000B091C7010196A11DB11D8093C401909314
:10359000C501A093C601B093C701BF91AF919F91A0
:1035A0008F910F900FBE0F901F9018950E948B0B5C
:1035B000F8942FEF87EA91E6215080409040E1F7A0
:1035C00000C0000087E090EBDC018093D80190936D
:1035D000D901A093DA01B093DB012CE088E190E0FF
:1035E0000FB6F894A895809360000FBE20936000FA
:1035F000FFCFCF92DF92EF92FF920F931F93CF9363
:10360000DF93C82E83E0D82E01E010E08D2D0E94BC
:103610009D077C01CBE0D0E098010C2E02C0220F68
:10362000331F0A94E2F72E213F21232B49F06C2F00
:103630007D2D80E00E94AF03C81202C081E007C068
:10364000219750F7DA948FEFD812E0CF80E0DF9126
:10365000CF911F910F91FF90EF90DF90CF90089541
:10366000CF93C82F8CE20E94F91A882321F08C2F67
:10367000CF910C94F91A80E0CF910895CF930E94D6
:10368000881C811102C00E94691CC5E6C15049F026
:103690000E9420078FE39CE90197F1F700C000002A
:1036A000F5CF89E20E94301B811111C18AE20E948C
:1036B000301B81110E94691C85E00E94301B811122
:1036C0000E94D61A0E94931C8093C20187E00E9438
:1036D000301B882399F18BE10E94301B882351F025
:1036E0009091C20191FB882780F921E0822780FB1D
:1036F00091F922C08EE00E94301B882351F09091F6
:10370000C20192FB882780F921E0822780FB92F991
:1037100013C080E10E94301B9091C201882341F0C8
:1037200093FB882780F921E0822780FB93F904C06E
:10373000892F809580FB90F99093C2018091C201FE
:103740000E94971C0E94A51C8093D60180EE0E94C7
:10375000301B882341F08091D601982F909590FBE3
:1037600080F98093D60189E30E94301B882359F0A9
:103770009091D60191FB882780F921E0822780FB78
:1037800091F99093D60182EE0E94301B882359F064
:103790009091D60192FB882780F921E0822780FB57
:1037A00092F99093D60186EE0E94301B882359F03F
:1037B0009091D60193FB882780F921E0822780FB36
:1037C00093F99093D60183EE0E94301B882359F021
:1037D0009091D60194FB882780F921E0822780FB15
:1037E00094F99093D60185E30E94301B882359F009
:1037F0009091D60195FB882780F921E0822780FBF4
:1038000095F99093D60181E30E94301B882359F0EB
:103810009091D60196FB882780F921E0822780FBD2
:1038200096F99093D60181E10E94301B882359F0CC
:103830009091D60197FB882780F921E0822780FBB1
:1038400097F99093D6018091D6010E94A91C80918E
:10385000D60187FB882780F980930C0187E20E94BC
:10386000301BC82F8EE10E94301B8111C2608FE196
:103870000E94301B8111C46080E20E94301B8111C4
:10388000C86081E20E94301B8111C06182E20E9407
:10389000301B8111C06283E20E94301B8111C06421
:1038A00084E20E94301B882311F0C06802C0CC2340
:1038B00029F08C2F0E94A01C6C2F03C00E949C1C1E
:1038C000682F70E080E090E0CF910C944E17CF917C
:1038D00008956DEE7EEF80E090E00E946D1E60E046
:1038E00082E090E00E945B1E60E083E090E00E9436
:1038F0005B1E60E084E090E00E945B1E60E085E07B
:1039000090E00E945B1E60E086E090E00C945B1EFD
:1039100080E090E00E94551E21E08D3E9E4F09F010
:1039200020E0822F089582E090E00C944D1E682FD5
:1039300082E090E00C945B1E83E090E00C944D1EBE
:10394000682F83E090E00C945B1E84E090E00C9480
:103950004D1E682F84E090E00C945B1E86E090E0A2
:103960000C944D1E682F86E090E00C945B1E8B310A
:1039700009F46AC008F58E3009F470C070F487301D
:1039800009F452C018F48630B9F134C0883009F413
:10399000A1C08B3009F49EC02DC0813109F479C0DB
:1039A00020F4803109F464C025C0863109F492C046
:1039B000893109F48FC01EC0853309F483C060F4D7
:1039C000873209F47FC020F48E3108F06DC012C038
:1039D000893209F477C00EC0833438F48A3308F092
:1039E00061C0883309F476C005C0833409F46AC025
:1039F000883461F080E008958091C201817F8E7FDC
:103A00008093C20181E08093C80108950E94501301
:103A10002FEF83ED90E3215080409040E1F700C00C
:103A200000000E94D61A56C09091C201892F80953D
:103A3000817080FB90F919F09660986027C0997F9B
:103A4000977F9093C20146C09091C20191FB882755
:103A500080F921E0822780FB91F913C09091C20187
:103A600092FB882780F921E0822780FB92F909C028
:103A70009091C20193FB882780F921E0822780FB87
:103A800093F99093C201882329F191609093C20128
:103A900008950E94501380910C0191E08927809332
:103AA0000C0118C027EC01C023EE280F61E070E084
:103AB00080E090E004C0660F771F881F991F2A9549
:103AC000D2F704C061E070E080E090E00E944E1701
:103AD0000E94501381E0089580E0089580E00895E9
:103AE000CF93C82F8091C801882319F0813049F005
:103AF0002EC0E0910D01F0910E018081823249F5D6
:103B000007C0E0910D01F0910E018081823249F4ED
:103B10008C2F0E946C1D811117C08C2F0E94B71C26
:103B200014C08C2F0E946E1D81110EC0C43149F04B
:103B300018F4CB3049F00FC0C93219F0C83321F066
:103B40000AC01092C80107C081E0817006C01092BF
:103B5000C80180E002C080E0F8CFCF9108950E94B4
:103B6000881C811102C00E94691C0E94AE1C8093B7
:103B7000D70180FF02C0869501C080E00C94FE0250
:103B80008091D701982F9695292F30E02830310564
:103B90004CF49F5F990F8170892B81608093D701CE
:103BA0000E94B21C8091D70186950C94FE028091F0
:103BB000D701982F969591F09158990F8170892B84
:103BC0008093D7018E7F91E009F490E08091D70136
:103BD00090FB80F98093D7010E94B21C8091D7019D
:103BE00086950C94FE028091D701982F909590FBBA
:103BF00080F98093D7010E94B21C8091D70180FF89
:103C000002C0869501C080E00C94FE023091D7017D
:103C1000232F26952F5F2F77822F90E03170099701
:103C20002CF4220F232B2093D70102C03093D7010D
:103C30008091D7018E7F91E009F490E08091D701C7
:103C400090FB80F98093D7010E94B21C8091D7012C
:103C500086950C94FE022091D701922F9695982775
:103C6000990F822F8170892B8093D7018E7F91E0ED
:103C700009F490E08091D70190FB80F98093D701FF
:103C80000E94B21C8091D70186950C94FE02EE0F23
:103C9000FF1F0590F491E02D0994F999FECF92BD94
:103CA00081BDF89A992780B50895A8E1B0E042E077
:103CB00050E00C94751E262FF999FECF92BD81BD60
:103CC000F89A019700B4021639F01FBA20BD0FB65A
:103CD000F894FA9AF99A0FBE08950196272F0E9438
:103CE0005C1E0C945B1EDC01CB01FC01F999FECF3C
:103CF00006C0F2BDE1BDF89A319600B40D92415074
:0A3D00005040B8F70895F894FFCF83
:103D0A00FFBB072608BE07F307BF070101AF01295A
:103D1A0039596943636F5F4F1F0F3379537F493FA7
:0E3D2A003639FD04C7048E043A0453046C04B9
:00000001FF
